:10000000D028FF3FFF3FFF3FAA2A0F398A0182070E
:100010003F3406345B344F3466346D347C340734FB
:100020007F34673477347C3439345E3479347134D6
:10003000050C06398A0182070000080001302428D7
:100040000230242800002728A800003008002808D3
:100050000339A80182070034013402340034110846
:1000600007398A018207A928AD28B228B728BC28F9
:10007000C128C628CB28110C9200920C120C1F39F3
:10008000820776287B287D287F2881288328852859
:10009000872889288B288D289228942896289828A4
:1000A0009A289C289E28A028A22807398A0182071E
:1000B0000134003400340034003408341034203467
:1000C00007398A01820700340134023404340834C9
:1000D00000340034003407398A01820701340234C5
:1000E0000434083410342034403480343F30A600C7
:1000F0006630A7000800063077285B3077284F303D
:100100007728663077286D3077287C30772807305D
:1001100077287F307728673077283F30A6006D300A
:10012000A700080006308E285B308E284F308E28BE
:1001300066308E286D308E287C308E2807308E28D1
:100140007F308E2867308E284030A6004030A700D0
:1001500008003F30A400A50008005B30A400063072
:10016000A50008006D30A4005B30A5000800073032
:10017000A4004F30A50008003F30A4006D30A5005A
:1001800008005B30A4007C30A50008006D30A4009E
:100190000730A50008000730A4007F30A500080044
:1001A0001F30860083161F308500013086008312C1
:1001B0006430810083168430810083120B118B160A
:1001C0008B17A801A901CD2AA8012230B822FF3936
:1001D000031DA9152130B822FF39031DA9142030B1
:1001E000B8229D00A821C1218A21FF39031926299F
:1001F0002913A913A91E17291D0303190D299D08E9
:10020000031D24290030A7000930A5003930A600BD
:100210000F30A400612229172629A9170030A70052
:10022000A600A500A400612294018E0126299D0844
:10023000031D24290030A700A4003930A6000F3088
:10024000A500612229172629A821C121051E861390
:10025000051A8617A91F3A298E08031D3A2904306A
:100260008E00140A073994005520A6001408602057
:10027000A500612285184B29291B4129A91F462960
:10028000542929132030A9066E23FA282911DA21CE
:10029000851C4829F328291BF4280518F42829155A
:1002A000DA21051C5129F328AA01AB016E23940120
:1002B00004308E00140A0F399400941D6629140826
:1002C00007396B202B05031D58296B2914086B2057
:1002D0002A05031D582914089D009D0A9D0AC12165
:1002E0008E0803195829851C8829051A7029861338
:1002F00032308E0005187029941D8329140807399F
:100300006B20AB04862914086B20AA047A23582991
:10031000A9132429182003390319003401390319BA
:100320009E299F30A91A11301D02031999299D0A8F
:10033000FF340030A91A00309D0098299D08031948
:10034000A3299D0398299F30A91A11309D0098294F
:10035000A91A08001D089E009F00291280301D0266
:10036000031C080090301D020318080030309F0263
:1003700029160800A91C08000611A122A1220615B1
:1003800008002918BA21061586152910A91ACF299F
:10039000022222308400E5211E08532208001D039A
:1003A0008F008F030F0D1E39B8229F00090AB82253
:1003B0009E00C829022220308400E5211F08532214
:1003C000861129190611291408000008F221840A4F
:1003D0000008F221000000008616000000008612CE
:1003E000861708008F000830900086138F0D0318C1
:1003F0008617000000000617000000000613900B8F
:10040000F52908005C30A91944301E02031C142A87
:10041000A430A919BC301E07A3006230A91984308A
:100420000318013EA2001F2A0830A91920301E0718
:10043000A3006230A91984300318013EA200A31B57
:10044000A20AA313A313A20C0318A317A21300302C
:1004500022382C301F02031C412A50301F02031C7B
:10046000392A1F08B03EA10073300318013EA000D6
:10047000482A1F08143EA10073300318013EA00053
:10048000482A1F08143EA10073300318013EA00043
:10049000A11BA00AA113A113A00C0318A117A0135C
:1004A00000302038080091002F203B208030A70426
:1004B000291AA404A91AA4041118602A0612612A90
:1004C00006160610000083160610000083120000B6
:1004D0008610703083220030832267308322240804
:1004E0008322250883222608832227088322831655
:1004F000000006100000831200008614000083161E
:10050000061483120800900008308F00900D031825
:100510008E2A0610831606108312912A831606145B
:100520008312000000008614000000008610000006
:100530008F0B862A00008614000000008610000041
:10054000080014309000FA308F008F0BA52A900B12
:10055000A32A08008C00030E8D006430013E0B11AD
:100560008E08031D8E030D0E83008C0E0C0E0900E9
:1005700089008316081483120808080088008B136A
:100580008316081555308900AA3089008814081E82
:10059000C72A081283128B1708003D308900B82241
:1005A0005E3C031DE02A3E308900B822783C031DE2
:1005B000E02A3F308900B822543C031DE02A042B76
:1005C00062308F0089010F08BE22890A0F08BE22FF
:1005D0008F0A8F0A890A891EE32A20308900883011
:1005E000BE2221308900FF30BE2222308900003037
:1005F000BE223D3089005E30BE22890A7830BE229C
:10060000890A5430BE22042B0518E4288518E428F2
:10061000AA23122336235A238623051C0D2B851C5F
:100620000D2BE4282230B8229300930923231820AD
:100630000339031D23238518172B22308900130843
:10064000BE226E2308009309031D2F2B0030A70044
:10065000A6003830A5003F30A40061220800003019
:10066000A700A6003E30A50073302C2B2130B82205
:1006700093009309472318200339031D4723851846
:100680003B2B213089001308BE226E2308009309FA
:10069000031D522B0030A7007C30A6007330A5004C
:1006A00054302C2B0030A7007C30A6007330A500FE
:1006B00066302C2B4030A7006D30A6007130A500AD
:1006C0004030A400612274232030B8229D2393007F
:1006D000203089001308BE226E230800851C6E2B73
:1006E000A122851C6E2B08008518742BA122851869
:1006F000742B0800051C7A2BA122051C7A2B0800FC
:100700000518802BA1220518802B080089016E2373
:100710008617090C0F39BD2374230908B8229D23BD
:10072000BE22890A86130908B8229D23BE22890A9F
:10073000203009050319872B08009D0053226E23E2
:100740001D08851C08008A21FF390319A02B1D08EC
:100750005322A02B0030A7003D30B822A6003E3027
:10076000B822A5003F30B822A40061223230C6234F
:100770000230BD233230C62308000520A5004030DA
:10078000A600A4000030A700612208008E000E0819
:10079000031DC72B0800FF3FFF3FFF3FFF3FFF3F09
:1007A000FF3FFF3FFF3FFF3FFF3FFF3FFF3FFF3F59
:1007B000FF3FFF3FFF3FFF3FFF3FFF3FFF3FFF3F49
:1007C000FF3FFF3FFF3FFF3FFF3FFF3FFF3FFF3F39
:1007D000FF3FFF3FFF3FFF3FFF3FFF3FFF3FFF3F29
:1007E000FF3FFF3FFF3FFF3FFF3FFF3FFF3FFF3F19
:1007F000FF3FFF3FFF3FFF3FFF3FFF3FFF3FFF3F09
:084000008C3F8E3F803F833F9F
:02400E00EB3F86
:00000001FF
